:100000000C940F020C9453020C9453020C94530260
:100010000C9453020C9453020C9453020C9453020C
:100020000C9453020C9453020C94070C0C94D90CAE
:100030000C9453020C9453020C9453020C945302EC
:100040000C9453020C94A3210C9453020C9453026D
:100050000C9453020C94321B0C9453020C945302D4
:100060000C9453020C9453020C9453020C945302BC
:100070000C9453020C9453020C9453020C945302AC
:100080000C9453020C9453020C9453020C9453029C
:100090000C9453020C9453020C9453020C9453028C
:1000A0000C9453020C9453020C945302460D680DA9
:1000B000560E680D560EAD0DD00D560E250E380E8F
:1000C0002411241161116111A411E211FB13FB131E
:1000D000FB11FB13FC12FC12CF13FB13FB13E613F3
:1000E00035002B00E000E1003A0000001E00140083
:1000F00004001D003B00E2001F001A0016001B0058
:100100003C00297120000700080006003D002A007D
:100110002100090017001900E300A90022000E00C9
:100120000A0005000000AA003E00310000002F0078
:100130000000A8003F000154000030000000AE00A5
:1001400023000D001C0013000000AB002400180069
:1001500011001000E700AC00250015000C0036006F
:1001600050002C0026000F00120037005100340010
:10017000270033000B0038005200E6002E002D004F
:100180002800E5004F00000001000100010001000F
:100190000100000001000100010001000100010058
:1001A0000100010001000100010001000100080040
:1001B0000700010001000100010015000900010015
:1001C0000100010001001700010001000000010012
:1001D0000100010000000100000001000100010019
:1001E000000001000000010001001C000B001100D4
:1001F00000000100010018000D00010001000100D5
:1002000001000C000E0001000100010001001200BD
:100210000F00010001000100010013003300010084
:1002200001000100010001000100010001000000C7
:1002300016034500720067006F0044006F007800ED
:10024000200045005A0000001603450072006700B8
:100250006F0044006F007800200045005A00000045
:100260000403090409026D00040100A0FA09040056
:10027000000103010100092111010001223F0007D3
:1002800005810308000A09040100010301020009B5
:100290002111010001224D000705820308000A090F
:1002A00004020001030000000921110100012236AF
:1002B000000705830308000A090403000103000086
:1002C00000092111010001223900070584031000F3
:1002D000011201100100000008EDFE0713010001EA
:1002E00002000105010906A101050719E029E7152A
:1002F0000025019508750181020508190129059558
:1003000005750191029501750391010507190029F1
:100310007715002501957875018102C005010980D6
:10032000A101850216010026B7001A01002AB700B4
:10033000751095018100C0050C0901A10185031606
:100340000100269C021A01002A9C02751095018169
:1003500000C005010902A1010901A1000509190157
:100360002905150025019505750181029501750383
:1003700081010501093009311581257F9502750834
:10038000810609381581257F950175088106050CC0
:100390000A38021581257F950175088106C0C005C0
:1003A000010906A101050719E029E71500250195B6
:1003B0000875018102950175088101050819012957
:1003C00005950575019102950175039101050719C0
:1003D0000029FF150025FF950675088100C0000063
:1003E000000000000000000000010204060A0F17D0
:1003F000202C3A4A5D71879DB3C7DAE9F5FCFFFC12
:10040000F5E9DAC7B39D87715D4A3A2C20170F0AC8
:10041000060402010000000000000000000011249A
:100420001FBECFEFDAE0DEBFCDBF04B603FE24C0AF
:100430008091EE019091EF01A091F001B091F10156
:100440008730904BA740B04BB9F41092EE01109258
:10045000EF011092F0011092F10114BE84B7877F72
:1004600084BF88E10FB6F89480936000109260001A
:100470000FBEE0E0FFE3099511E0A0E0B1E0E4ED9C
:10048000F6E402C005900D92A433B107D9F711E04C
:10049000A4E3B1E001C01D92AE3EB107E1F70E94B6
:1004A0004B090C9468230C94000008950895609102
:1004B000B1017091B2018091B3019091B4010E9499
:1004C0005E1A56985E9825982D9826982E9827980B
:1004D0002F98813011F4259A2D9A08950C94570283
:1004E00056985E9825982D9826982E9827982F989C
:1004F0008FEF90E0909389008093880090938B0019
:1005000080938A0090938D0080938C00259A2D9A79
:100510002FEF80E792E0215080409040E1F700C04B
:100520000000269A2E9A2FEF80E792E0215080401B
:100530009040E1F700C00000279A2F9A2FEF80E744
:1005400092E0215080409040E1F700C000002598E3
:100550002D982FEF80E792E0215080409040E1F706
:1005600000C0000026982E982FEF80E792E02150DF
:1005700080409040E1F700C0000027982F985698DF
:100580005E9825982D9826982E9827982F9808954C
:1005900089EA8093800089E08093810024982C98D8
:1005A0003F988AB18F748AB96E98479A8BB1806BE5
:1005B0008BB9769A0E9470020C94560280E2809366
:1005C00000018091340181110EC00E942D0381E051
:1005D000809334012FEF83ED90E3215080409040D1
:1005E000E1F700C0000080E40E9433038093000123
:1005F00081112EC00E945D0380930001811128C0EB
:100600000E945D0380930001811122C08FE30E944C
:100610005D038093000181111BC00E94550380E49B
:100620000E94330380930001811112C08CE00E946C
:100630005D038093000181110BC00E945D038093D4
:100640000001811105C08FE30E945D0380930001CA
:100650000E9455038091000108951092B9008AE02C
:100660008093B800089594EA9093BC009091BC00E8
:1006700097FFFCCF9091B900987F983021F090318E
:1006800011F081E008958093BB0084E88093BC0062
:100690008091BC0087FFFCCF8091B900887F8831B2
:1006A00011F0803471F780E0089584E98093BC00F4
:1006B0008091BC0084FDFCCF08958093BB0084E84A
:1006C0008093BC008091BC0087FFFCCF9091B90063
:1006D000987F81E0983209F480E0089584E880935F
:1006E000BC008091BC0087FFFCCF8091BB000895C7
:1006F00080910001811115C080E40E943303809332
:10070000000181110CC082E10E945D038093000111
:10071000811105C08FEF0E945D03809300010E944C
:10072000550384B1807F84B985B1807F85B98AB152
:10073000837F8AB98BB1837F8BB93E9846980895A1
:100740000E94DE02809300010E94780380B38C70C7
:1007500080BB81B3836F81BBA6E3B1E0E4E4F1E049
:100760008EE08E0F11921D928E13FCCF0C94C80256
:10077000BF92CF92DF92EF92FF920F931F93CF938E
:10078000DF9380910001882379F0809135018F5F9C
:1007900080933501811108C00E94DE028093000120
:1007A000811102C00E94700206E311E0C0E0D0E0B7
:1007B000DD24D39482E0C82EEE24E394F12CC730DC
:1007C000D10500F580910001811164C080E40E9490
:1007D000330380930001811112C082E10E945D0306
:1007E0008093000181110BC0C7010C2E01C0880F3E
:1007F0000A94EAF780950E945D03809300010E94AD
:10080000550348C0CA30A1F028F4C83059F0C930A7
:1008100061F005C0CC3089F070F0CD3089F0209ABD
:10082000289810C0219A29980DC0229A2A980AC0A7
:10083000239A2B9807C0529A01C0539A5B9802C022
:100840003E9A469890EA9A95F1F79FB1799902C03D
:1008500082E001C080E091709D25982B7C9902C0B8
:1008600084E001C080E0892B7D9902C038E001C09E
:1008700030E0832B7E9902C020E101C020E0822B72
:100880009FB19095991F9927991F9295990F907EE6
:10089000892B0FC080910001811149C080E40E9422
:1008A000330380930001882379F1B12C0E94550312
:1008B0008B2DF8019081981719F08083C092010167
:1008C0000E94780321960F5F1F4FCE30D10509F0AB
:1008D00076CF80910101882361F1815080930101DD
:1008E000882339F08FE99FE00197F1F700C00000FD
:1008F00020C0A4E4B1E0E6E3F1E0CF01825F919192
:100900009D938E13FCCF15C083E10E945D038093FD
:1009100000018111CACF81E40E943303809300015A
:100920008111C3CF0E946E03B82EB094BFCF80E078
:10093000C0CF0E946E0281E0DF91CF911F910F9195
:10094000FF90EF90DF90CF90BF900895E82FF0E0F8
:10095000EC5BFE4F808108950895089596E0799F9D
:10096000F001112494E5899FE00DF11D1124E60F9B
:10097000F11DEE0FFF1FE052FF4F859194910895F6
:10098000880F991FFC01E05AF040859194910895D9
:10099000880F991FFC01E052FF4F859194910895B3
:1009A0000F931F93CF93DF93EC018115904350F584
:1009B000C11580E2D80708F0B3C0CB3BD10590F455
:1009C000C83AD10508F05AC0C53AD10508F04BC065
:1009D000C430D10508F0BBC1219709F0B5C101E0D1
:1009E00010E0F5C1CF3FD10511F008F0B0C1C03F14
:1009F000D10508F092C0CE01805E9109089708F4F5
:100A0000A6C1A2C1C11591E5D907A8F4C23020E55D
:100A1000D20708F09EC0C11580E5D80709F485C04B
:100A200008F091C0C11520E4D20708F08DC1DD2780
:100A30008E01106CCCC1C11580E8D80758F4C115DF
:100A400090E7D90708F07CC1C11520E6D20708F469
:100A500022C17AC1C11580E9D80708F075C1DF70DD
:100A60008E01106AB4C1C53AD10509F472C1C63A03
:100A7000D10509F071C102E810E4A9C1C83AD10555
:100A800009F46DC1C93AD10509F46CC1CA3AD1055E
:100A900009F46BC1CB3AD10509F46AC1CC3AD1054E
:100AA00009F469C1CD3AD10509F468C1C03BD1054B
:100AB00009F467C1CE3AD10509F466C1CF3AD10530
:100AC00009F465C1C13BD10509F464C1C23BD1053C
:100AD00009F463C1C33BD10509F462C1C43BD1052C
:100AE00009F461C1C53BD10509F460C1C63BD1051C
:100AF00009F45FC1C73BD10509F45EC1C83BD1050C
:100B000009F45DC1C93BD10509F45CC1CA3BD105FB
:100B100009F45BC100E014E45AC18E01106557C1AD
:100B2000CE019F700E94C80453C10E941F149FEF02
:100B300024E38CE0915020408040E1F700C00000A9
:100B40000E94571B44C18091CD0181608093CD01EB
:100B50003EC10E94001D811102C00E94E61C0E943D
:100B60001D1D90E09093EE018093ED01C23090E561
:100B7000D90721F48091ED01816086C0C43020E561
:100B8000D20721F48091ED0182607EC0C63080E5FD
:100B9000D80721F48091ED01846076C0C83090E5DB
:100BA000D90719F48091ED0127C0CA3020E5D2079A
:100BB00021F48091ED01806167C0CC3080E5D807D9
:100BC00021F48091ED0180625FC0CE3090E5D907BD
:100BD00021F48091ED01806457C0C03120E5D20737
:100BE00021F48091ED0180684FC0C23180E5D807C3
:100BF00029F48091ED018460886046C0C33090E59F
:100C0000D90721F48091ED018E7F3EC0C53020E5EB
:100C1000D20721F48091ED018D7F36C0C73080E589
:100C2000D80721F48091ED018B7F2EC0C93090E56B
:100C3000D90719F48091ED0126C0CB3020E5D20709
:100C400021F48091ED018F7E1FC0CD3080E5D80763
:100C500021F48091ED018F7D17C0CF3090E5D90749
:100C600021F48091ED018F7B0FC0C13120E5D207C7
:100C700021F48091ED018F7707C0C331D04531F465
:100C80008091ED018B7F877F8093ED018091ED0155
:100C90000E94211D9CC08D2F99278F70992781302C
:100CA0009105D9F49E012370332702C0880F991F44
:100CB0002A95E2F79C688E0144E0000F111F4A95C7
:100CC000E1F700271370802B912B53E0CC0FDD1F31
:100CD0005A95E1F7C076DD272FC08230910531F4B7
:100CE000DC2FCC278E01016F106A71C08330910513
:100CF00069F4CE018370992701E010E002C0000F73
:100D0000111F8A95E2F7C8019C680FC0049709F08B
:100D10005EC0CE018370992701E010E002C0000F91
:100D2000111F8A95E2F7C8019A6823E0CC0FDD1FF6
:100D30002A95E1F7C07ED7708C010C2B1D2B47C084
:100D4000DF708E01106243C000E010E040C08E01F1
:100D50003EC001E810E43BC003E810E438C002EEF6
:100D600014E435C009EE14E432C00AEE14E42FC0D6
:100D700005EB14E42CC006EB14E429C007EB14E4E3
:100D800026C00CEC14E423C00DEC14E420C003E8EE
:100D900015E41DC00AE815E41AC002E915E417C0FD
:100DA00004E915E414C001E216E411C003E216E4FC
:100DB0000EC004E216E40BC005E216E408C006E229
:100DC00016E405C007E216E402C00AE216E4C80110
:100DD000DF91CF911F910F91089596E0799FF001D7
:100DE000112494E5899FE00DF11D1124E60FF11DFA
:100DF000EE0FFF1FE052FF4F85919491803E9105C9
:100E0000E0F4803C910558F58133910509F46FC0F9
:100E100048F48932910509F463C08A32910509F4D6
:100E20006DC072C089339105E9F082389105D1F027
:100E30008533910509F44DC067C0833E910581F16A
:100E400038F4803E9105B9F0823E9105D9F05CC03E
:100E5000863E910561F1873E9105A1F155C00E9442
:100E6000C00408952091ED0120FD02C021FF4CC077
:100E700080EE90E049C08091ED0180FFF9CF89E3D9
:100E800090E042C08091ED0182FF0EC08091ED01A3
:100E900084FF03C080E090E037C083EE90E034C070
:100EA0008091ED0182FFF2CF82EE90E02DC0809123
:100EB000ED0183FF0BC08091ED0184FDEBCF87EE48
:100EC00090E022C08091ED0183FFF5CF86EE90E0A7
:100ED0001BC08091ED0185FF07C089E290E014C03E
:100EE0008091ED0185FFF9CF85E390E00DC0809101
:100EF000ED0186FF07C08AE290E006C08091ED0117
:100F000086FFF9CF81E390E00E94D0040895089510
:100F10000C948707809162010895CF93DF9300D0EE
:100F20001F92CDB7DEB79C018091E401843019F5A2
:100F300093E099833B832A839093E9008FEF90910C
:100F4000E800815095FD06C095ED9A95F1F70000F7
:100F50008111F5CF8091E80085FF0DC040E050E0A1
:100F600063E070E0CE0101960E94F7098091E800ED
:100F70008E778093E8000F900F900F90DF91CF91C4
:100F80000895CF93DF9300D01F92CDB7DEB72091A5
:100F9000E401243021F522E029839B838A8383E0C6
:100FA0008093E9008FEF9091E800815095FD06C095
:100FB00095ED9A95F1F700008111F5CF8091E80049
:100FC00085FF0DC040E050E063E070E0CE01019687
:100FD0000E94F7098091E8008E778093E8000F90D7
:100FE0000F900F90DF91CF9108952091E40124306C
:100FF000F1F422E02093E9002FEF3091E800215036
:1010000035FD06C035ED3A95F1F700002111F5CF19
:101010002091E80025FF0BC040E050E065E070E063
:101020000E94F7098091E8008E778093E800089588
:10103000CF93DF93EC019091E401943009F046C026
:1010400080910C018823D9F080910D018823B9F09B
:101050009093E9008FEF9091E800815095FD06C0D4
:1010600095E19A95F1F700008111F5CF8091E800A4
:1010700085FF2CC040E050E060E170E017C081E0E7
:101080008093E9008FEF9091E800815095FD06C0B4
:1010900095ED9A95F1F700008111F5CF8091E80068
:1010A00085FF14C040E050E068E070E0CE010E948F
:1010B000F7098091E8008E778093E80080E1FE01D7
:1010C000A2E5B1E001900D928A95E1F7DF91CF9111
:1010D00008958091E301811109C00E948C0B0E9448
:1010E000E90B8091E20084608093E2000895109201
:1010F000E301089508950C9490210E94ED1A0E9436
:1011000096210E948F0E0C94880742E061EC81E0EA
:101110000E94060B42E061EC82E00E94060B42E076
:1011200061EC83E00E94060B42E161EC84E00C94E8
:10113000060B8091E601833009F455C030F481300C
:1011400071F0823009F48EC008958A3009F47AC0B3
:101150008B3009F460C0893009F09CC020C08091B8
:10116000E501813A09F096C08091E800877F80937D
:10117000E8008091E9019091EA01892B21F460E176
:1011800082E591E003C060E080E090E070E00E94C2
:10119000420A8091E8008B778093E800089580915F
:1011A000E501813209F076C08091E9019091EA0170
:1011B000009719F0039709F06DC08091E800877FD0
:1011C0008093E8008091E80082FD05C08091E401F1
:1011D0008111F8CF5FC08091F1008093620180910E
:1011E000E8008B7753C08091E501813A09F052C045
:1011F0008091E9019091EA01892B09F04BC080911F
:10120000E800877F8093E8008091E80080FFFCCFB2
:1012100080910C0136C08091E5018132D9F5809131
:10122000E9019091EA01892BA9F58091E800877F77
:101230008093E8000E943B0B8091E70180930C01B2
:101240000C941F148091E501813221F58091E80012
:10125000877F8093E8000E943B0B8091E801809398
:10126000630108958091E501813AA1F48091E8003D
:10127000877F8093E8008091E80080FFFCCF809119
:1012800063018093F1008091E8008E778093E800FD
:101290000C943B0B089584B7877F84BF88E10FB619
:1012A000F89480936000109260000FBE90E080E898
:1012B0000FB6F89480936100909361000FBE0E9476
:1012C000DE0E0E948C0B0E94E90B8091E20084608C
:1012D0008093E20078940E946F0E0E94E00E82E0FC
:1012E00091E00E948A0E0E947E218091E401853067
:1012F00069F40E94AE1A8091E2018823B1F30E9442
:10130000D91A882391F30E94E109EFCF0E94E60EDB
:10131000ECCF292F332723303105C9F064F4213075
:10132000310581F02230310509F043C08DE690E0AF
:1013300024E632E042C021323105F1F0223231059B
:1013400041F137C082E190E021ED32E036C09927CB
:101350008130910541F08230910541F0892B49F5AA
:10136000E0E6F2E005C0E8E4F2E002C0E0E3F2E02B
:10137000849190E09F0121C06430D8F4E62FF0E022
:10138000EE0FFF1FEE5DFE4F2081318189E090E07E
:1013900014C0643070F470E0FB01EE0FFF1FE65ED6
:1013A000FE4F20813181FB01EA5EFE4F808190E09B
:1013B00004C080E090E020E030E0FA013183208337
:1013C000089580E189BD82E189BD09B400FEFDCFA9
:1013D0008091D8008F7D8093D8008091E00082605A
:1013E0008093E0008091E00081FDFCCF0895CF92D2
:1013F000DF92EF92FF920F931F93CF93DF93EC0155
:101400008B016A010E945A0B811133C0C114D104AF
:1014100039F0F60180819181081B190BC80FD91F83
:10142000E12CF12C0115110519F18091E80085FDE1
:1014300016C08091E8008E778093E800C114D10433
:1014400049F0F60180819181E80EF91EF182E08277
:1014500085E00FC00E945A0B882321F30AC08991AE
:101460008093F10001501109FFEFEF1AFF0ADACF64
:1014700080E0DF91CF911F910F91FF90EF90DF906F
:10148000CF9008952091EB013091EC01261737079A
:1014900048F06115710539F42091E8002E7720930A
:1014A000E80001C0B90140E061157105A9F1209182
:1014B000E401222309F443C0253009F442C02091FD
:1014C000E80023FD40C02091E80022FD32C02091B9
:1014D000E80020FFE9CF4091F3002091F20030E0D6
:1014E000342BFC01CF016115710559F0283031050D
:1014F00040F481918093F100615071092F5F3F4F5B
:10150000F1CF41E02830310509F040E02091E800BA
:101510002E772093E800C8CF4111C9CF0AC080912F
:10152000E401882361F0853061F08091E80083FD5B
:101530000AC08091E80082FFF2CF80E0089582E047
:10154000089583E0089581E008952091EB013091A2
:10155000EC012617370748F06115710539F4209121
:10156000E8002E772093E80001C0B901FC0120E0DB
:101570006115710591F18091E401882309F440C05F
:10158000853009F43FC08091E80083FD3DC0809123
:10159000E80082FD2FC08091E80080FFE9CF209114
:1015A000F3008091F20090E0922B6115710559F0E3
:1015B0008830910540F424912093F10031966150D8
:1015C00071090196F2CF21E0089709F020E080919F
:1015D000E8008E778093E800CBCF2111CCCF0AC0F2
:1015E0008091E401882361F0853061F08091E8000A
:1015F00083FD0AC08091E80082FFF2CF80E0089569
:1016000082E0089583E0089581E00895982F97304F
:1016100058F59093E900981739F07091EC002091FB
:10162000ED005091F00003C0242F762F50E021FFF1
:1016300019C03091EB003E7F3093EB003091ED000C
:101640003D7F3093ED003091EB0031603093EB0043
:101650007093EC002093ED005093F0002091EE0089
:1016600027FF07C09F5FD3CF8F708093E90081E091
:10167000089580E008958091E50187FF11C0809171
:10168000E80082FD05C08091E4018111F8CF11C00E
:101690008091E8008B770BC08091E401882349F0AA
:1016A0008091E80080FFF8CF8091E8008E778093EA
:1016B000E80008952091E4003091E50095E640911E
:1016C000EC00842F817040FF22C08091E80080FDF3
:1016D0001CC08091E401882391F0853091F08091C5
:1016E000EB0085FD10C04091E4005091E5004217E9
:1016F000530729F39A01915011F784E0089582E08D
:10170000089583E0089581E0089580E00895409170
:10171000E80042FFDECF08950E94FA0B0E94020CFF
:10172000E0EEF0E0808181608083E8EDF0E0808190
:101730008F77808319BCA7EDB0E08C918E7F8C935E
:1017400080818F7E80831092E30108950F931F9311
:10175000CF93DF930E94FA0B0E94020CC8EDD0E0F9
:1017600088818F77888388818068888388818F7D4E
:10177000888319BC1092E4011092E0011092E201FA
:101780001092E10100EE10E0F80180818B7F8083F0
:1017900088818160888342E060E080E00E94060BDF
:1017A000E1EEF0E080818E7F8083E2EEF0E08081E8
:1017B00081608083808188608083F80180818E7F52
:1017C0008083888180618883DF91CF911F910F9101
:1017D0000895E8EDF0E080818F7E8083E7EDF0E012
:1017E00080818160808384E082BF81E08093E30117
:1017F0000C94A60BE8EDF0E080818E7F8083109240
:10180000E20008951092DA001092E10008951F920C
:101810000F920FB60F9211242F933F934F935F9324
:101820006F937F938F939F93AF93BF93EF93FF93A8
:101830008091E10082FF0BC08091E20082FF07C02F
:101840008091E1008B7F8093E1000E946E0E809179
:10185000DA0080FF1FC08091D80080FF1BC08091FC
:10186000DA008E7F8093DA008091D90080FF0DC06E
:1018700080E189BD82E189BD09B400FEFDCF81E030
:101880008093E4010E94690805C019BC1092E4012C
:101890000E9477088091E10080FF19C08091E200EA
:1018A00080FF15C08091E2008E7F8093E2008091DE
:1018B000E20080618093E2008091D8008062809392
:1018C000D80019BC85E08093E4010E947B088091D8
:1018D000E10084FF30C08091E20084FF2CC080E1F1
:1018E00089BD82E189BD09B400FEFDCF8091D80099
:1018F0008F7D8093D8008091E1008F7E8093E100FE
:101900008091E2008F7E8093E2008091E20081600E
:101910008093E2008091E001882311F084E007C009
:101920008091E30087FD02C081E001C083E08093E5
:10193000E4010E947D088091E10083FF29C080912D
:10194000E20083FF25C08091E100877F8093E10062
:1019500082E08093E4011092E0018091E1008E7FAB
:101960008093E1008091E2008E7F8093E20080917D
:10197000E20080618093E20042E060E080E00E944B
:10198000060B8091F00088608093F0000E947A0836
:10199000FF91EF91BF91AF919F918F917F916F9147
:1019A0005F914F913F912F910F900FBE0F901F901D
:1019B00018951F920F920FB60F9211242F933F93F9
:1019C0004F935F936F937F938F939F93AF93BF9347
:1019D000CF93DF93EF93FF93C091E900CF70809195
:1019E000EC00D82FD17080FDD0E81092E9008091F2
:1019F000F000877F8093F00078940E941D0D109274
:101A0000E9008091F00088608093F000CD2BCF70CA
:101A1000C093E900FF91EF91DF91CF91BF91AF911A
:101A20009F918F917F916F915F914F913F912F91F6
:101A30000F900FBE0F901F9018951F93CF93DF93B9
:101A4000CDB7DEB7AA970FB6F894DEBF0FBECDBFF5
:101A5000E5EEF1E088E08E0F9091F10091938E1306
:101A6000FBCF0E9499088091E80083FF1FC18091FD
:101A7000E5019091E601492F50E04A30510508F008
:101A800015C1FA01EA5AFF4F0C941823803881F0EF
:101A9000823809F00BC18091E9018F708093E900D1
:101AA0008091EB0085FB882780F91092E90006C041
:101AB0008091E1019091E201911182609091E800A2
:101AC000977F9093E8008093F1001092F100C8C0D6
:101AD000282F2D7F09F0EAC0882319F0823061F0A9
:101AE000E5C08091E701813009F0E0C0933009F052
:101AF00080E08093E2012BC08091E701811127C033
:101B00008091E9018F7009F4D1C08093E9002091A0
:101B1000EB0020FF1CC0933021F48091EB00806229
:101B200014C09091EB0090619093EB0021E030E0C5
:101B3000A90102C0440F551F8A95E2F74093EA00BD
:101B40001092EA008091EB0088608093EB00109285
:101B5000E9008091E800877F86C08111A7C01091BD
:101B6000E7011F778091E3008078812B8093E30069
:101B70008091E800877F8093E8000E943B0B809172
:101B8000E80080FFFCCF8091E30080688093E30051
:101B9000111102C082E001C083E08093E40186C09D
:101BA0008058823008F082C08091E7019091E8016E
:101BB0008C3D53E0950779F583E08A838AE2898337
:101BC0004FB7F894DE01139620E03EE051E2E32F98
:101BD000F0E050935700E49120FF03C0E295EF70CE
:101BE0003F5FEF708E2F90E0EA3010F0C79601C093
:101BF000C0968D939D932F5F243149F74FBF8091FD
:101C0000E800877F8093E8006AE270E0CE010196E9
:101C10000E94420A14C0AE014F5F5F4F6091E9011C
:101C20000E948909BC01892B09F440C09091E80009
:101C3000977F9093E80089819A810E94A50A8091FC
:101C4000E8008B778093E80031C0803879F5809187
:101C5000E800877F8093E8008091E0018093F100A5
:101C60008091E8008E778093E8000E943B0B1EC0B5
:101C700081111CC09091E7019230C0F48091E8007E
:101C8000877F8093E8009093E0010E943B0B809156
:101C9000E001811106C08091E30087FD02C081E070
:101CA00001C084E08093E4010E9485088091E800EF
:101CB00083FF0AC08091E800877F8093E8008091CD
:101CC000EB0080628093EB00AA960FB6F894DEBF1B
:101CD0000FBECDBFDF91CF911F9108950895CF938F
:101CE0008091E4018823A1F0C091E900CF70909128
:101CF000EC00892F817090FD80E8C82B1092E900DC
:101D00008091E80083FD0E941D0DCF70C093E90013
:101D1000CF91089590936901809368010895E091AF
:101D20006801F0916901309721F00190F081E02D78
:101D3000099480E00895E0916801F091690130977D
:101D400021F00280F381E02D09940895E09168016B
:101D5000F0916901309721F00480F581E02D09941C
:101D6000089520916601309167018217930771F001
:101D70009093670180936601E0916801F091690199
:101D8000309721F00680F781E02D09940895209185
:101D90006401309165018217930771F0909365019A
:101DA00080936401E0916801F0916901309721F01E
:101DB0000084F185E02D0994089508950C94DD0EBA
:101DC0000E94F31A0E94A0030C94B91BCF92DF92D9
:101DD000EF92FF920F931F93CF93DF93CDB7DEB7B0
:101DE0002B970FB6F894DEBF0FBECDBF0E94B8038D
:101DF0008BE6C82E81E0D82E00E010E0E02E802F88
:101E00000E94A604F60141916F01F42EF826B1F468
:101E10000F5F1F4F0E30110589F78FEF89838A837B
:101E20001B820E94FC1A8160782F9D838C834981DC
:101E30005A816B818D810E94890F40C09091CD01A4
:101E400091FF04C08B870E94AC048B8520E030E0BA
:101E50004F2D50E0922FBA01022E02C07595679562
:101E60000A94E2F760FF24C02E83EF8221E030E085
:101E7000690102C0CC0CDD1C9A95E2F790E08C2140
:101E80009D21892B09F420E028870E94FC1A81609B
:101E9000782F9A8789874E815F8168858A850E941D
:101EA000890FF801E559FE4F8081C826C08206C01F
:101EB0002F5F3F4F2630310569F6AACF0E94A01E42
:101EC00010916A010E948F0E1817A1F00E948F0EC8
:101ED00080936A012B960FB6F894DEBF0FBECDBF7C
:101EE000DF91CF911F910F91FF90EF90DF90CF90F6
:101EF0000C9488072B960FB6F894DEBF0FBECDBFAB
:101F0000DF91CF911F910F91FF90EF90DF90CF90D5
:101F10000895CF93DF93CDB7DEB72B970FB6F89424
:101F2000DEBF0FBECDBF4F83588769877A878B8707
:101F3000DE01119686E0FD0111928A95E9F785E0B0
:101F4000FE01379601900D928A95E1F749815A81F9
:101F50006B817C818D819E810E94B9162B960FB674
:101F6000F894DEBF0FBECDBFDF91CF9108950895E5
:101F7000CF93882309F4C2C0C82F823859F40E9435
:101F80008F0E81FDBBC089E30E9462190E942F1A47
:101F900089E30CC0833879F40E948F0E80FDAEC0B7
:101FA00083E50E9462190E942F1A83E50E94A419FA
:101FB000CF910C942F1A843859F40E948F0E82FD11
:101FC0009DC087E40E9462190E942F1A87E4EECF19
:101FD0008CEF8C0F813A48F48C2F0E94E320811102
:101FE0008DC08C2F0E946219E3CF80E28C0F883065
:101FF00048F4C77081E001C0880FCA95EAF70E94D3
:10200000E819D6CF8BE58C0F833078F4C53A29F0E8
:10201000C63A31F083E890E005C081E890E002C064
:1020200082E890E0CF910C94B10E88E58C0F83315B
:1020300008F064C0C83A39F1C93A41F1CA3A49F1E5
:10204000CB3A51F1CC3A59F1CD3A61F1C03B69F14B
:10205000CE3A71F1CF3A79F1C13B81F1C23B89F1BE
:10206000C33B91F1C43B99F1C53BA1F1C63BA9F13A
:10207000C73BB1F1C83BB9F1C93BC1F1CA3BC9F19A
:1020800080E090E038C082EE90E035C089EE90E0CC
:1020900032C08AEE90E02FC085EB90E02CC086EB3A
:1020A00090E029C087EB90E026C08CEC90E023C044
:1020B0008DEC90E020C083E891E01DC08AE891E0BB
:1020C0001AC082E991E017C084E991E014C081E26E
:1020D00092E011C083E292E00EC084E292E00BC075
:1020E00085E292E008C086E292E005C087E292E0D5
:1020F00002C08AE292E0CF910C94C70ECF9108956E
:10210000882309F44BC0823859F40E948F0E81FF56
:1021100045C089E30E9462190E942F1A89E30CC00E
:10212000833871F40E948F0E80FF38C083E50E94CF
:1021300062190E942F1A83E50E94A4190C942F1A89
:10214000843859F40E948F0E82FF28C087E40E94D1
:1021500062190E942F1A87E4EFCF9CEF980F913AF3
:1021600058F390E2980F983050F4877091E001C0D6
:10217000990F8A95EAF7892F0E94EE19DFCF9BE528
:10218000980F933020F480E090E00C94B10E885AC0
:10219000833120F480E090E00C94C70E08958823EA
:1021A00021F00E94E8190C942F1A0895882321F039
:1021B0000E94EE190C942F1A0895BF92CF92DF92CD
:1021C000EF92FF920F931F93CF93DF9300D000D035
:1021D00000D0CDB7DEB725E0FC01DE0111960190FD
:1021E0000D922A95E1F7FC01D080118102812581B1
:1021F00022952F7043815481452B09F4FCC21F3F67
:1022000021F4FFEFDF1609F4F6C27C012E830E9451
:10221000B70FD9821A8369817A81802F0E945E1953
:10222000182FB92E0E9413190E94DA172E8100234D
:1022300019F00E94051A2E81EB2DE295EF70F0E067
:10224000E05AFF4F0C9418238B2D807F9B2D9F709D
:10225000F92E882319F0F29480EFF822002389F0F8
:10226000FF2009F475C280E2810F883020F48F2DA1
:102270000E94E81903C08F2D0E94F8190E942F1A9E
:1022800067C2812F0E948010FF2009F4B4C2105E43
:102290008F2D183018F40E94EE1902C00E94FE190A
:1022A00026960FB6F894DEBF0FBECDBFDF91CF915B
:1022B0001F910F91FF90EF90DF90CF90BF900C9403
:1022C0002F1A3B2D307F8B2D8F70303211F082957D
:1022D000807F112319F0113021F12CC00023B9F0B7
:1022E000222309F4A0C1213009F09DC126960FB622
:1022F000F894DEBF0FBECDBFDF91CF911F910F913C
:10230000FF90EF90DF90CF90BF900C94181A22238B
:1023100019F0213009F46FC28E830E941B1A8E813E
:1023200096C1002321F0223008F065C27CC1211142
:1023300062C28DC1002321F0222309F474C108C2B6
:10234000222309F484C119C22B2D269526952370CA
:1023500030E02115310521F021303105D1F04BC29B
:10236000002321F0812F9B2D937002C080E090E02C
:1023700026960FB6F894DEBF0FBECDBFDF91CF918A
:102380001F910F91FF90EF90DF90CF90BF900C9432
:10239000B10E002321F0812F9B2D937002C080E0AD
:1023A00090E026960FB6F894DEBF0FBECDBFDF914A
:1023B000CF911F910F91FF90EF90DF90CF90BF9042
:1023C0000C94C70E812F002319F00E94A81D02C093
:1023D0000E94101E26960FB6F894DEBF0FBECDBF2A
:1023E000DF91CF911F910F91FF90EF90DF90CF90F1
:1023F000BF900C94951E8B2D837009F07BC001114A
:10240000FAC1812F829586958770880F880F912F4A
:102410009F70C92ED12CE12CF12C082E04C0CC0CBD
:10242000DD1CEE1CFF1C0A94D2F714FF12C04FE013
:1024300050E060E070E004C0440F551F661F771F36
:102440008A95D2F7CB01BA016095709580959095E9
:1024500003C060E070E0CB012B2D269526952370FC
:10246000422F50E042305105D9F04330510569F117
:102470006C297D298E299F294130510551F12696DD
:102480000FB6F894DEBF0FBECDBFDF91CF911F9185
:102490000F91FF90EF90DF90CF90BF900C940118B8
:1024A0006C297D298E299F2926960FB6F894DEBFC8
:1024B0000FBECDBFDF91CF911F910F91FF90EF9095
:1024C000DF90CF90BF900C941D180E940118C70197
:1024D000B60126960FB6F894DEBF0FBECDBFDF91D2
:1024E000CF911F910F91FF90EF90DF90CF90BF9011
:1024F0000C94E517002319F08B2D817001C086958F
:10250000882309F478C1812F829586958770880F7A
:10251000880F912F9F70C92ED12CE12CF12C082E01
:1025200004C0CC0CDD1CEE1CFF1C0A94D2F714FF77
:1025300012C04FE050E060E070E004C0440F551F4F
:10254000661F771F8A95D2F7CB01BA016095709507
:102550008095909503C060E070E0CB012B2D26950F
:1025600026952370422F50E042305105D9F0433078
:10257000510569F16C297D298E299F29413051052A
:1025800051F126960FB6F894DEBF0FBECDBFDF9196
:10259000CF911F910F91FF90EF90DF90CF90BF9060
:1025A0000C94DB186C297D298E299F2926960FB65D
:1025B000F894DEBF0FBECDBFDF91CF911F910F9179
:1025C000FF90EF90DF90CF90BF900C94F7180E948F
:1025D000DB18C701B60126960FB6F894DEBF0FBE12
:1025E000CDBFDF91CF911F910F91FF90EF90DF90C2
:1025F000CF90BF900C94BF18103FD1F118F4103E4B
:1026000050F4A1C0123F09F463C008F44CC0133F5A
:1026100009F473C098C01F708B2D8F710023A1F037
:102620000E945818812F26960FB6F894DEBF0FBE71
:10263000CDBFDF91CF911F910F91FF90EF90DF9071
:10264000CF90BF900C94CF100E947918812F2696BE
:102650000FB6F894DEBF0FBECDBFDF91CF911F91B3
:102660000F91FF90EF90DF90CF90BF900C94D61019
:102670000023A9F02111BFC08B2D8F7126960FB6B4
:10268000F894DEBF0FBECDBFDF91CF911F910F91A8
:10269000FF90EF90DF90CF90BF900C949E18223067
:1026A00008F0A9C0E9CF0023A9F08B2D8F712696E1
:1026B0000FB6F894DEBF0FBECDBFDF91CF911F9153
:1026C0000F91FF90EF90DF90CF90BF900C9458182F
:1026D000002359F38B2D8F7126960FB6F894DEBF29
:1026E0000FBECDBFDF91CF911F910F91FF90EF9063
:1026F000DF90CF90BF900C947918002399F08B2D28
:102700008F7126960FB6F894DEBF0FBECDBFDF9156
:10271000CF911F910F91FF90EF90DF90CF90BF90DE
:102720000C94431826960FB6F894DEBF0FBECDBFAB
:10273000DF91CF911F910F91FF90EF90DF90CF909D
:10274000BF900C9439180023A9F0222309F4ADCFCF
:10275000812F26960FB6F894DEBF0FBECDBFDF9156
:10276000CF911F910F91FF90EF90DF90CF90BF908E
:102770000C94B80F222309F4ADCF812F26960FB603
:10278000F894DEBF0FBECDBFDF91CF911F910F91A7
:10279000FF90EF90DF90CF90BF900C9480104B2D66
:1027A0004F70612FC7010E94550226960FB6F8940C
:1027B000DEBF0FBECDBFDF91CF911F910F91FF9074
:1027C000EF90DF90CF90BF900C945D174B2D4F7022
:1027D000612FC70126960FB6F894DEBF0FBECDBF9E
:1027E000DF91CF911F910F91FF90EF90DF90CF90ED
:1027F000BF900C94AD0426960FB6F894DEBF0FBEC2
:10280000CDBFDF91CF911F910F91FF90EF90DF909F
:10281000CF90BF9008950E94051A0E94151A0E9439
:10282000DA190E942F1A0E94461F0E94951E80E00E
:1028300090E00E94B10E80E090E00C94C70E0E94E0
:10284000F5190C940B140E945319292F22952F70FF
:1028500030E02C3031054CF42A3031056CF4225034
:1028600031092230310588F407C02C30310549F098
:102870002F30310531F009C0803E48F0803F29F407
:1028800006C093FB882780F9089580E0089581E0D1
:102890000895CF93DF9300D000D01F92CDB7DEB75D
:1028A0000F900F900F900F900F90DF91CF910895A0
:1028B000CF93DF9300D000D000D0CDB7DEB72696FF
:1028C0000FB6F894DEBF0FBECDBFDF91CF91089554
:1028D0001F93CF93DF93C091790116E080917A0125
:1028E000C81799F0D0E01C9FF0011D9FF00D112436
:1028F000E558FE4F408151816281738184819581C9
:102900000E9458142196C770E9CFDF91CF911F9193
:1029100008954091AB015091AC016091AD0170916F
:10292000AE018091AF019091B0010C945814809148
:10293000B00182958F7009F054C08091AD01882359
:1029400009F44FC080917901A0917A016091AB01A7
:102950007091AC014091AE015091AF01B6E08A1781
:1029600009F43FC090E041155105C1F17F3F11F4DA
:102970006F3FA1F1B89FF001B99FF00D1124E55808
:10298000FE4F218172132AC02081621327C0228149
:10299000211124C0238134812417350710F42150DC
:1029A0003109241B350B283C3105C0F42091B001BE
:1029B0002F7020612093B00126E0289FF001299F0D
:1029C000F00D1124E058FE4F80818F70806180836C
:1029D0008BEA91E00E94DD100C94681401968770D8
:1029E000BECF0895CF92DF92EF92FF920F931F9385
:1029F000CF93DF93CDB7DEB762970FB6F894DEBF03
:102A00000FBECDBF8C0185E0F801DE011D9601905F
:102A10000D928A95E1F7D8014C9111965C9111972E
:102A200012966C9112971396CD90DC90149730917A
:102A3000AB017091AC018091AE019091AF01009714
:102A400009F46BC17F3F19F43F3F09F466C1E09080
:102A5000AD01EE2009F4C0C02091B001C816D9061E
:102A600028F0F601E81BF90BCF0104C08095909582
:102A70008C0D9D1DFF24F394883C910578F0F12C7A
:102A8000207F09F0C6C07C2DD98AC88A89890E9416
:102A900049148BEA91E00E94DD10B1C0822F807F43
:102AA00009F046C0751314C0341312C0611110C070
:102AB0002F7020612093B0010E9489148BEA91E06D
:102AC0000E94DD108091B001D80115968C932EC024
:102AD000CD2819F15F3F11F44F3FF9F0F62E611147
:102AE0001CC08091790120917A0136E0821709F4A7
:102AF0005AC090E0389FF001399FF00D1124E5583D
:102B0000FE4F7181571306C07081471303C0728155
:102B1000711103C001968770E9CFF62E662309F480
:102B200018C18091B00181608093B001F12C11C176
:102B3000751308C0341306C0611104C08091B00140
:102B4000D801C3C04D875E878D859E856A8B0E94A4
:102B500023146A898823E1F16623D1F12091B00121
:102B6000822F82958F7090E0029774F08091AB0174
:102B70009091AC0198878F831986DB86CA862C8753
:102B8000CE0107960E94DD1086E0F801ABEAB1E0C5
:102B900001900D928A95E1F70E9497140E94891482
:102BA000FF24F394D6C04D875E878D859E850E9455
:102BB0005319292F22952F7030E0223031050CF067
:102BC000BCC09F7009F0B6C0805E883008F4C1C0F8
:102BD000C8010E94DD10E4CFC816D90608F453C01E
:102BE000F601E81BF90BCF01883C910508F450C0B1
:102BF000F12C7C2DD98AC88A89890E944914EBEA74
:102C0000F1E086E0DF011D928A95E9F70E948914C0
:102C1000A0C0751314C0341312C0611110C080918C
:102C2000B001F8018583C8010E94DD1086E0EBEA5F
:102C3000F1E0DF011D928A95E9F7FE2C8AC04D87ED
:102C40005E878D859E856A8B0E9423146A898823FE
:102C500009F4BECF662309F4BBCF2091B001822FC7
:102C600082958F7090E002970CF48ECF8091AB012B
:102C70009091AC019A8389831B82DD82CC822E8362
:102C8000CE0101967FCF809590958C0D9D1DACCF88
:102C9000F62E662309F49CCF75132EC034132CC076
:102CA0002091B00120FD1FC0822F82958F70D9F036
:102CB000D80115962C9315978F3049F08F5F982F78
:102CC0009295907F822F8F70892B15968C93C801D7
:102CD0000E94DD1086E0F801ABEAB1E001900D92B0
:102CE0008A95E1F793CF86E0F801ABEAB1E0019075
:102CF0000D928A95E1F72DC04D875E878D859E8563
:102D00000E942314811140CF8091B0018160809393
:102D1000B001C8010E94DD101CC0662309F458CF21
:102D20004D875E878D859E850E942314882309F434
:102D30004FCF2ACF811148CF0CC0243031050CF081
:102D400047CF9F7009F440CFF8019581907F09F03B
:102D50003BCF8F2D62960FB6F894DEBF0FBECDBF6E
:102D6000DF91CF911F910F91FF90EF90DF90CF9067
:102D700008951F93CF93DF93CDB7DEB72C970FB68F
:102D8000F894DEBF0FBECDBF4F83588769877A871F
:102D90008B879C87CE0107960E94F214882369F0E6
:102DA0008F8198852A853B85232BF1F19F3F09F080
:102DB00063C08F3F09F060C037C086E0FE013796E0
:102DC000DE01119601900D928A95E1F76F81788569
:102DD000EA85FB85309741F17F3F11F46F3F21F188
:102DE00020917A0130E0C9010196877099274091BE
:102DF000790150E08417950709F447C069837A8305
:102E0000FD83EC8396E0929FD001939FB00D112437
:102E1000A558BE4FFE01319601900D929A95E1F7AB
:102E200080937A010E94681416E080917901909154
:102E30007A018917C1F1189FC001112485589E4F4E
:102E40000E94F214882379F1E09179011E9FF0012C
:102E50001124E558FE4F4081518162817381848144
:102E600095810E9458148091790190E001968770B5
:102E7000992780937901D9CF4F81588569857A85C3
:102E80008B859C850E945814CFCF0E941F141092EE
:102E90007A0110927901EBEAF1E086E0DF011D9200
:102EA0008A95E9F7C1CF2C960FB6F894DEBF0FBE16
:102EB000CDBFDF91CF911F910895EF92FF920F93B5
:102EC0001F93CF93DF938C01892B09F46CC0F12CF5
:102ED000EE24E394E8012196F8018491843740F4CC
:102EE000843008F051C0813081F0823019F15BC02C
:102EF000853709F444C0A8F19CE7980F903708F093
:102F000052C08F770E94801041C00E5F1F4FFE019C
:102F1000C49180E28C0F883048F4C7708E2D01C0B8
:102F2000880FCA95EAF70E94081A14C08C2F0E94D5
:102F3000B80F2DC00E5F1F4FFE01C49180E28C0FB1
:102F4000883058F4C7708E2D01C0880FCA95EAF7F3
:102F50000E940E1A0E942F1A1AC08C2F0E948010F5
:102F600016C00E5F1F4FFE01C491CC2381F08FE984
:102F70009FE00197F1F700C00000C150F6CF0E5F4F
:102F80001F4FFE01F49003C00E94B80F8E018F2DD9
:102F9000882309F49FCFEFE9FFE03197F1F700C0F4
:102FA00000008150F5CFDF91CF911F910F91FF90DD
:102FB000EF90089508956093B5017093B6018093E2
:102FC000B7019093B8010C940B140F931F930091C9
:102FD000B5011091B6012091B7013091B801DC0123
:102FE000CB01802B912BA22BB32B8093B501909317
:102FF000B601A093B701B093B8011F910F910C9443
:103000000B140F931F930091B5011091B6012091FD
:10301000B7013091B801DC01CB0180239123A223B9
:10302000B3238093B5019093B601A093B701B093F9
:10303000B8011F910F910C940B140F931F930091E3
:10304000B5011091B6012091B7013091B801DC01B2
:10305000CB0180279127A227B3278093B5019093B6
:10306000B601A093B701B093B8011F910F910C94D2
:103070000B141092B1011092B2011092B301109290
:10308000B4010C940B1441E050E060E070E004C027
:10309000440F551F661F771F8A95D2F74093B101E1
:1030A0005093B2016093B3017093B4010C940B146C
:1030B00041E050E060E070E004C0440F551F661F1F
:1030C000771F8A95D2F78091B1019091B201A091BA
:1030D000B301B091B401482B592B6A2B7B2B409341
:1030E000B1015093B2016093B3017093B4010C9499
:1030F0000B1441E050E060E070E004C0440F551F45
:10310000661F771F8A95D2F7409550956095709508
:103110008091B1019091B201A091B301B091B4013D
:10312000482359236A237B234093B1015093B20172
:103130006093B3017093B4010C940B1441E050E020
:1031400060E070E004C0440F551F661F771F8A952A
:10315000D2F78091B1019091B201A091B301B091E9
:10316000B401482759276A277B274093B101509320
:10317000B2016093B3017093B4010C940B140F93DC
:103180001F930091B1011091B2012091B3013091D0
:10319000B401DC01CB01802B912BA22BB32B8093AC
:1031A000B1019093B201A093B301B093B4011F9108
:1031B0000F910C940B140F931F930091B101109178
:1031C000B2012091B3013091B401DC01CB01802325
:1031D0009123A223B3238093B1019093B201A093D2
:1031E000B301B093B4011F910F910C940B140F9382
:1031F0001F930091B1011091B2012091B301309160
:10320000B401DC01CB0180279127A227B32780934B
:10321000B1019093B201A093B301B093B4011F9197
:103220000F910C940B140895CF92DF92EF92FF92BE
:103230000F931F93CF93DF938C01C090B501D09073
:10324000B601E090B701F090B8018091B101909182
:10325000B201A091B301B091B401C82AD92AEA2AD7
:10326000FB2ACFE1D0E0D701C6010C2E04C0B695F1
:10327000A795979587950A94D2F780FF06C0B80165
:103280008C2F0E94ED06019721F4219760F780E0D2
:1032900001C08C2FDF91CF911F910F91FF90EF9084
:1032A000DF90CF900895CF93DF93EC010E94141923
:1032B000BE010E94ED06DF91CF910895CB010E94DF
:1032C0005319089590910C01992321F090910D01CB
:1032D000911109C020910E0130910F01F901329630
:1032E0009FEF40E01FC0982F9695969596959F303A
:1032F00050F5E0910E01F0910F01E90FF11D87707B
:1033000021E030E0A90102C0440F551F8A95E2F781
:10331000CA019181892B818308959F3F39F04F5FC6
:103320004E3041F051915813F8CF0DC05111F7CFE5
:10333000942FF5CF9F3F39F0F901E90FF11D97FD6B
:10334000FA9582830895089590910C01992321F0B4
:1033500090910D01911109C020910E0130910F0142
:10336000F9013296205F3F4F1FC0982F9695969592
:1033700096959F30F0F4E0910E01F0910F01E90F66
:10338000F11D877021E030E0A90102C0440F551FF4
:103390008A95E2F7CA0180959181892381830895F6
:1033A0003196E217F30729F090819813F9CF108234
:1033B000F7CF089581E090E0E0910E01F0910F01C8
:1033C000E80FF91F1082019680319105A9F7089541
:1033D0009091CC01892B8093CC0108958095909198
:1033E000CC0189238093CC0108951092CC010895DB
:1033F0009091CB01892B8093CB010895809590917A
:10340000CB0189238093CB0108951092CB010895BD
:103410009091CA01892B8093CA010895809590915B
:10342000CA0189238093CA0108951092CA010895A0
:103430008093B90108951092B901089580910E0109
:1034400090910F01FC0131969C01205F3F4F80E07D
:10345000919191118F5FE217F307D1F70895E091F1
:103460000E01F0910F018091CC018083E0910E015B
:10347000F0910F0190818091CB01892B8083E091A5
:103480000E01F0910F0190818091CA01892B8083F8
:103490008091B901882361F0E0910E01F0910F0154
:1034A0009081892B80830E941E1A81111092B9018C
:1034B00080910E0190910F010C949B0ECF92DF92A0
:1034C000EF92FF926C01EE24FF24C114D104E104B9
:1034D000F10421F0C701B60120E101C020E0C72EB0
:1034E000D82EE92EFF24C114D104E104F10419F00F
:1034F000285FC701B6016B017C0154E0F694E794A4
:10350000D794C7945A95D1F7C114D104E104F104BA
:1035100019F02C5FC701B6016B017C0142E0F69403
:10352000E794D794C7944A95D1F7C114D104E10424
:10353000F10419F02E5FC701B601DC01CB01B6958D
:10354000A79597958795892B8A2B8B2B09F02F5F51
:10355000822FFF90EF90DF90CF9008958091E4014B
:10356000843021F11092CE0120E488E190E00FB682
:10357000F894A895809360000FBE2093600080E0CF
:103580000E94880783B7817F846083BF83B781608F
:1035900083BF7894889583B78E7F83BF88E10FB609
:1035A000F89480936000109260000FBE0895089513
:1035B0000895CF930E94D71A0E94B8030E94D81A88
:1035C000C0E08C2F0E94A604811104C0CF5FCE30D2
:1035D000C1F701C081E0CF9108950E941F140E949D
:1035E0008F0E0C94880782E084BD93E095BD9AEF1E
:1035F00097BD80936E0008952FB7F8948091CF0106
:103600009091D001A091D101B091D2012FBF089526
:10361000CF92DF92EF92FF920F931F932FB7F89400
:103620004091CF015091D0016091D1017091D201B0
:103630002FBF6A017B01EE24FF248C0120E030E0E3
:10364000C016D106E206F30610F4415051099A0162
:10365000281B390BC9011F910F91FF90EF90DF904C
:10366000CF9008951F920F920FB60F9211248F934F
:103670009F93AF93BF938091CF019091D001A09180
:10368000D101B091D2010196A11DB11D8093CF014E
:103690009093D001A093D101B093D201BF91AF918B
:1036A0009F918F910F900FBE0F901F9018950E94C1
:1036B0008C0BF8942FEF87EA91E6215080409040E0
:1036C000E1F700C0000087E090EBDC018093EE01A1
:1036D0009093EF01A093F001B093F1019CE088E199
:1036E0000FB6F894A895809360000FBE9093600089
:1036F000FFCFEF92FF920F931F93CF93DF93D82FBB
:10370000C0E08C2F0E94A60400E010E0E82EF12C0F
:10371000C701002E02C0959587950A94E2F780FDB7
:1037200006C00F5F1F4F0630110591F709C0602FCB
:103730007C2F80E00E94AE04D813F3CF81E004C058
:10374000CF5FCE30F1F680E0DF91CF911F910F91E6
:10375000FF90EF900895CF93C82F8CE20E94791BC1
:10376000882321F08C2FCF910C94791B80E0CF918E
:103770000895CF930E94001D811102C00E94E61C93
:10378000C5E6C15049F00E94B8038FE39CE9019758
:10379000F1F700C00000F5CF89E20E94AB1B811158
:1037A00013C18AE20E94AB1B81110E94E61C85E0D6
:1037B0000E94AB1B81110E94571B0E940B1D80931E
:1037C000CD0187E00E94AB1B8823A9F18BE10E9409
:1037D000AB1B882351F08091CD0181FB222720F97A
:1037E00091E0922790FB81F90EC08EE00E94AB1B06
:1037F000882361F08091CD0182FB222720F991E09E
:10380000922790FB82F98093CD0115C080E10E9440
:10381000AB1B9091CD01882341F093FB222720F927
:1038200081E0822780FB93F904C0892F809580FB7B
:1038300090F99093CD018091CD010E940F1D0E94BF
:103840001D1D8093ED0180EE0E94AB1B882341F08B
:103850008091ED01982F909590FB80F98093ED0178
:1038600089E30E94AB1B882359F08091ED0181FB15
:10387000222720F991E0922790FB81F98093ED01B6
:1038800082EE0E94AB1B882359F08091ED0182FBF0
:10389000222720F991E0922790FB82F98093ED0195
:1038A00086EE0E94AB1B882359F08091ED0183FBCB
:1038B000222720F991E0922790FB83F98093ED0174
:1038C00083EE0E94AB1B882359F08091ED0184FBAD
:1038D000222720F991E0922790FB84F98093ED0153
:1038E00085E30E94AB1B882359F08091ED0185FB95
:1038F000222720F991E0922790FB85F98093ED0132
:1039000081E30E94AB1B882359F08091ED0186FB77
:10391000222720F991E0922790FB86F98093ED0110
:1039200081E10E94AB1B882359F08091ED0187FB58
:10393000222720F991E0922790FB87F98093ED01EF
:103940008091ED010E94211D8091ED0187FB882768
:1039500080F980930D0187E20E94AB1BC82F8EE196
:103960000E94AB1B8111C2608FE10E94AB1B8111D1
:10397000C46080E20E94AB1B8111C86081E20E949A
:10398000AB1B8111C06182E20E94AB1B8111C0623E
:1039900083E20E94AB1B8111C06484E20E94AB1BD6
:1039A000882311F0C06802C0CC2329F08C2F0E941C
:1039B000181D6C2F03C00E94141D682F70E080E05A
:1039C00090E0CF910C94DB17CF9108956DEE7EEFD0
:1039D00080E090E00E94522360E082E090E00E944C
:1039E000402360E083E090E00E94402360E084E0B8
:1039F00090E00E94402360E085E090E00C9440233A
:103A000080E090E00E943A2321E08D3E9E4F09F035
:103A100020E0822F089582E090E00C943223682FFA
:103A200082E090E00C94402383E090E00C943223F9
:103A3000682F83E090E00C94402384E090E00C94A5
:103A40003223682F84E090E00C9440238091D501CC
:103A500080FF0BC06091130185E0689FB0011124C5
:103A600075956795759567952BC081FF09C0609125
:103A7000130185E0689FB00111247595679520C0FA
:103A800082FF07C06091130185E0689FB001112497
:103A900017C09091D6019923D1F060911201961729
:103AA00088F72091130185E0289F90011124929FAF
:103AB000A001939F500D112470E0CA010E940423BD
:103AC0006038710540F46115710539F002C065E098
:103AD00070E0862F08958FE7089581E00895809122
:103AE000D50180FF08C06091110170E07595679560
:103AF0007595679521C081FF06C06091110170E046
:103B00007595679519C082FF04C06091110170E03E
:103B100010C09091D6019923C1F0609110019617C1
:103B2000A0F780911101899FC001112470E00E94CB
:103B300004236038710528F46115710521F0862F82
:103B400008958FE7089581E0089561E070E0F4CF73
:103B5000803F21F40E94261D819504C0813F29F4F5
:103B60000E94261D8093D9010895823F21F40E946E
:103B7000261D819504C0833F29F40E94261D809351
:103B8000D8010895893F19F40E946F1D05C08A3F2E
:103B900031F40E946F1D81958093DA0108958B3F67
:103BA00021F40E946F1D819504C08C3F29F40E946E
:103BB0006F1D8093DB010895843F21F48091D7012C
:103BC000816017C0853F21F48091D701826011C0C8
:103BD000863F21F48091D70184600BC0873F21F498
:103BE0008091D701886005C0883F31F48091D7016A
:103BF00080618093D70108958D3F21F48091D50194
:103C000081600BC08E3F21F48091D501826005C098
:103C10008F3F29F48091D50184608093D501089568
:103C2000803F39F48091D90187FF6CC01092D9018F
:103C300069C0813F29F48091D9011816BCF362C094
:103C40009091D801823F29F497FF5CC01092D8016F
:103C500059C0833F19F41916CCF354C0893F41F47D
:103C60008091DA0118160CF04DC01092DA014AC0AA
:103C70008A3F29F48091DA0187FF44C0F6CF8B3F59
:103C800039F48091DB0187FF3DC01092DB013AC01F
:103C90008C3F29F48091DB011816BCF333C0843FBC
:103CA00021F48091D7018E7F17C0853F21F4809148
:103CB000D7018D7F11C0863F21F48091D7018B7F82
:103CC0000BC0873F21F48091D701877F05C0883FD3
:103CD00031F48091D7018F7E8093D70113C08D3F3F
:103CE00021F48091D5018E7F0BC08E3F21F480910D
:103CF000D5018D7F05C08F3F29F48091D5018B7F41
:103D00008093D5018091D80181110EC08091D90195
:103D100081110AC08091DA01811106C08091DB0116
:103D2000811102C01092D601089587ED91E00E94A2
:103D3000A60E0E94FC1A9093D4018093D30108959B
:103D40001F93CF93DF938091D3019091D4010E9470
:103D5000081BAC019091D601992321F02091140108
:103D600030E006C0209115018AE0289F90011124BF
:103D70004217530708F486C08091D801C091D90139
:103D8000D091DA011091DB01811107C0C11176C019
:103D9000D11174C0111172C075C09F3F19F09F5F9F
:103DA0009093D601181624F40E94261D8093D80102
:103DB0008091D80187FF05C00E94261D81958093C0
:103DC000D8011C1624F40E94261D8093D9018091ED
:103DD000D90187FF05C00E94261D81958093D901D6
:103DE0006091D801662339F1C091D901CC2319F132
:103DF000772767FD7095872F972F0E94152223E361
:103E000033E343E35FE30E9479220E94E22160935F
:103E1000D8016C2F772767FD7095872F972F0E9409
:103E2000152223E333E343E35FE30E9479220E94F8
:103E3000E2216093D9011D1624F40E946F1D809326
:103E4000DA018091DA0187FF05C00E946F1D81951C
:103E50008093DA01111624F40E946F1D8093DB0118
:103E60008091DB0187FF05C00E946F1D81958093C3
:103E7000DB01DF91CF911F910C94951E9F3F09F0BC
:103E80008ECF96CFDF91CF911F910895E7EDF1E0AE
:103E900085E0DF011D928A95E9F71092D601109214
:103EA000D5010895833081F128F4813059F08230B2
:103EB000D1F00895853009F449C0B8F1863009F48D
:103EC00056C0089580911501262F30E0280F311D2E
:103ED0002F3F310524F4680F6093150108958FEF8B
:103EE00080931501089580911401262F30E0280F4A
:103EF000311D2F3F310524F4680F6093140108959C
:103F00008FEF80931401089580911301262F30E0E4
:103F1000280F311D2F3F310524F4680F60931301E2
:103F200008958FEF80931301089580911201262F39
:103F300030E0280F311D2F3F310524F4680F6093C6
:103F4000120108958FEF809312010895809111015D
:103F5000262F30E0280F311D2F3F310524F4680F44
:103F60006093110108958FEF80931101089580915E
:103F70001001262F30E0280F311D2F3F310524F48A
:103F8000680F6093100108958FEF809310010895DA
:103F9000833011F128F4813049F0823091F0089596
:103FA000853081F120F18630C1F1089580911501AD
:103FB000681720F4861B809315010895109215014F
:103FC000089580911401681720F4861B80931401D2
:103FD000089510921401089580911301681720F438
:103FE000861B809313010895109213010895809108
:103FF0001201681720F4861B809312010895109215
:104000001201089580911101681720F4861B809396
:1040100011010895109211010895809110016817FF
:1040200020F4861B809310010895109210010895CA
:104030000F931F938D3109F46BC008F03FC08E3091
:1040400009F47FC0C0F4873009F469C068F4863091
:1040500009F0B1C08091CD01817F8E7F8093CD0129
:1040600081E08093DD01A8C0883009F4A2C08B30C4
:1040700009F49FC0A0C0863109F49BC078F4803158
:1040800009F472C0813109F096C00E941F1490910A
:104090000D0181E0892780930D018BC0893109F4DE
:1040A00088C08B3109F087C08091CD0181FB222728
:1040B00020F991E0922790FB81F94CC0853309F4F7
:1040C00070C048F4873209F46CC008F459C08932D2
:1040D00009F467C070C0833438F48A3308F04EC0E6
:1040E000883309F466C067C0833409F45AC0883441
:1040F00009F061C00E941F140FEF13ED20E301507F
:1041000010402040E1F700C000000E94571B51C042
:104110000E949C210E948F0E0E9488074AC09091A5
:10412000CD01892F8095817080FB90F929F09660F0
:1041300098609093CD0140C0997F977F9093CD0177
:1041400038C08091CD0182FB222720F991E092278F
:1041500090FB82F98093CD01992359F18091CD0193
:1041600081608093CD0125C08091CD0183FB222702
:1041700020F991E0922790FB83F9ECCF895301C09D
:104180008D5141E050E060E070E08A019B0104C085
:10419000000F111F221F331F8A95D2F7C901B801E2
:1041A00004C061E070E080E090E00E94DB170E94B4
:1041B0001F1481E001C080E01F910F91089580E0FD
:1041C000089580E00895CF93C82F8091DD0181305C
:1041D00079F018F08230E9F187C0E0910E01F0919A
:1041E0000F018081813169F0823209F07FC009C0FE
:1041F000E0910E01F0910F018081813111F0823246
:1042000061F48C2F0E94DF20811104C08C2F0E944A
:1042100018201DC081E090E01AC08C2F0E94E12080
:10422000811114C0C43179F048F4CB3079F0C03139
:1042300009F060C082E08093DD0108C0C93219F046
:10424000C83321F057C01092DD0154C081E0817065
:1042500053C0C93289F118F5C43171F1A8F4C730DF
:1042600009F046C08AE08093150194E1909314010F
:1042700093E0909313018093120188E080931101E1
:1042800088E28093100134C0CE51C63088F5EC2FFF
:10429000F0E0E65DFE4F80818093DC0129C0CE34E2
:1042A000E9F020F4CB3421F56AE013C0C13579F090
:1042B000C235F1F461E00DC08091DC01882319F072
:1042C0001092DC0115C081E08093DD0115C061E032
:1042D00006C08091DC010E94521F0AC06AE08091F2
:1042E000DC010E94C81F04C01092DD0180E004C000
:1042F00081E002C080E0ABCFCF910895E1E8F0E02B
:104300008081886080838081816080838FB7F8940A
:1043100093E09093890090ED909388008FBF08956B
:10432000EFE6F0E08081826080830895EFE6F0E0C0
:1043300080818D7F80830895EFE6F0E0908182E0B8
:104340008927808308951F920F920FB60F92112430
:104350002F933F934F935F936F937F938F939F938D
:10436000AF93BF93EF93FF938091DE019091DF01B4
:1043700001969093DF018093DE01811103C082E0FA
:104380000E948807E091DF01E695E695F0E0E252B1
:10439000FC4FE4918091DE018E1303C080E00E9407
:1043A0008807FF91EF91BF91AF919F918F917F917E
:1043B0006F915F914F913F912F910F900FBE0F9092
:1043C0001F90189504D06894B1118DC0089570D0D5
:1043D00088F09F5790F0B92F9927B751A0F0D1F0EE
:1043E000660F771F881F991F1AF0BA95C9F712C078
:1043F000B13081F077D0B1E0089574C0672F782F85
:104400008827B85F39F0B93FCCF3869577956795E3
:10441000B395D9F73EF490958095709561957F4F4F
:104420008F4F9F4F0895E89409C097FB3EF49095F5
:104430008095709561957F4F8F4F9F4F9923A9F07D
:10444000F92F96E9BB279395F6958795779567950C
:10445000B795F111F8CFFAF4BB0F11F460FF1BC050
:104460006F5F7F4F8F4F9F4F16C0882311F096E9E3
:1044700011C0772321F09EE8872F762F05C0662391
:1044800071F096E8862F70E060E02AF09A95660F4A
:10449000771F881FDAF7880F9695879597F9089503
:1044A00057FD9058440F551F59F05F3F71F04795E5
:1044B000880F97FB991F61F09F3F79F087950895CA
:1044C000121613061406551FF2CF4695F1DF08C0E9
:1044D000161617061806991FF1CF86957105610506
:1044E00008940895E894BB2766277727CB0197F9AE
:1044F00008950BD078C069D028F06ED018F09523BD
:1045000009F05AC05FC01124EECFCADFA0F3959F17
:10451000D1F3950F50E0551F629FF001729FBB27AA
:10452000F00DB11D639FAA27F00DB11DAA1F649F56
:104530006627B00DA11D661F829F2227B00DA11D09
:10454000621F739FB00DA11D621F839FA00D611D8F
:10455000221F749F3327A00D611D231F849F600DB0
:10456000211D822F762F6A2F11249F5750408AF0E9
:10457000E1F088234AF0EE0FFF1FBB1F661F771F75
:10458000881F91505040A9F79E3F510570F014C00C
:10459000AACF5F3FECF3983EDCF38695779567955D
:1045A000B795F795E7959F5FC1F7FE2B880F911D93
:1045B0009695879597F9089597F99F6780E870E039
:1045C00060E008959FEF80EC089500240A94161689
:1045D000170618060906089500240A9412161306F1
:1045E000140605060895092E0394000C11F488237F
:1045F00052F0BB0F40F4BF2B11F460FF04C06F5F9B
:104600007F4F8F4F9F4F089597FB072E16F400940E
:1046100007D077FD09D00E941E2307FC05D03EF489
:10462000909581959F4F0895709561957F4F08955E
:10463000EE0FFF1F0590F491E02D0994AA1BBB1B00
:1046400051E107C0AA1FBB1FA617B70710F0A61B92
:10465000B70B881F991F5A95A9F780959095BC01B3
:10466000CD010895F999FECF92BD81BDF89A9927A1
:1046700080B50895A8E1B0E042E050E00C945A23E0
:10468000262FF999FECF92BD81BDF89A019700B40B
:10469000021639F01FBA20BD0FB6F894FA9AF99AAB
:1046A0000FBE08950196272F0E9441230C944023AA
:1046B000DC01CB01FC01F999FECF06C0F2BDE1BDE2
:1046C000F89A319600B40D9241505040B8F70895D1
:0446D000F894FFCF8C
:1046D40020028A071808F507C1078D070101BA01EE
:1046E40028080A03140A3F4D36399F0352031C035A
:1046F400E30276028F02A802C10201020304050646
:044704000708090099
:00000001FF
